 jncrypto

 Timestamp is 15a77d7b (reproducible build file hash)

 Preferred load address is 0000000180000000

 Start         Length     Name                   Class
 0001:00000000 00006370H .text$mn                CODE
 0001:00006370 00000036H .text$mn$00             CODE
 0001:000063a6 00000092H .text$x                 CODE
 0002:00000000 000001b8H .idata$5                DATA
 0002:000001b8 00000038H .00cfg                  DATA
 0002:000001f0 00000008H .CRT$XCA                DATA
 0002:000001f8 00000008H .CRT$XCZ                DATA
 0002:00000200 00000008H .CRT$XIA                DATA
 0002:00000208 00000008H .CRT$XIZ                DATA
 0002:00000210 00000008H .CRT$XPA                DATA
 0002:00000218 00000008H .CRT$XPZ                DATA
 0002:00000220 00000008H .CRT$XTA                DATA
 0002:00000228 00000008H .CRT$XTZ                DATA
 0002:00000230 00000000H .gehcont$y              DATA
 0002:00000230 00000000H .gfids$y                DATA
 0002:00000230 000010d0H .rdata                  DATA
 0002:00001300 00000000H .rdata$CastGuardVftablesA DATA
 0002:00001300 00000000H .rdata$CastGuardVftablesC DATA
 0002:00001300 00000064H .rdata$voltmd           DATA
 0002:00001364 000002bcH .rdata$zzzdbg           DATA
 0002:00001620 00000008H .rtc$IAA                DATA
 0002:00001628 00000008H .rtc$IZZ                DATA
 0002:00001630 00000008H .rtc$TAA                DATA
 0002:00001638 00000008H .rtc$TZZ                DATA
 0002:00001640 00000470H .xdata                  DATA
 0002:00001ab0 000009c0H .edata                  DATA
 0002:00002470 00000078H .idata$2                DATA
 0002:000024e8 00000018H .idata$3                DATA
 0002:00002500 000001b8H .idata$4                DATA
 0002:000026b8 00000448H .idata$6                DATA
 0003:00000000 00000040H .data                   DATA
 0003:00000040 00000940H .bss                    DATA
 0004:00000000 00000444H .pdata                  DATA
 0005:00000000 00000060H .rsrc$01                DATA
 0005:00000060 000003a0H .rsrc$02                DATA

  Address         Publics by Value              Rva+Base               Lib:Object

 0000:00000000       __AbsoluteZero             0000000000000000     <absolute>
 0000:00000000       ___safe_se_handler_count   0000000000000000     <absolute>
 0000:00000000       ___safe_se_handler_table   0000000000000000     <absolute>
 0000:00000000       __arm64x_extra_rfe_table   0000000000000000     <absolute>
 0000:00000000       __arm64x_extra_rfe_table_size 0000000000000000     <absolute>
 0000:00000000       __arm64x_native_entrypoint 0000000000000000     <absolute>
 0000:00000000       __arm64x_redirection_metadata 0000000000000000     <absolute>
 0000:00000000       __arm64x_redirection_metadata_count 0000000000000000     <absolute>
 0000:00000000       __dynamic_value_reloc_table 0000000000000000     <absolute>
 0000:00000000       __enclave_config           0000000000000000     <absolute>
 0000:00000000       __guard_check_icall_a64n_fptr 0000000000000000     <absolute>
 0000:00000000       __guard_eh_cont_count      0000000000000000     <absolute>
 0000:00000000       __guard_eh_cont_table      0000000000000000     <absolute>
 0000:00000000       __guard_fids_count         0000000000000000     <absolute>
 0000:00000000       __guard_fids_table         0000000000000000     <absolute>
 0000:00000000       __guard_iat_count          0000000000000000     <absolute>
 0000:00000000       __guard_iat_table          0000000000000000     <absolute>
 0000:00000000       __guard_longjmp_count      0000000000000000     <absolute>
 0000:00000000       __guard_longjmp_table      0000000000000000     <absolute>
 0000:00000000       __hybrid_auxiliary_iat     0000000000000000     <absolute>
 0000:00000000       __hybrid_auxiliary_iat_copy 0000000000000000     <absolute>
 0000:00000000       __hybrid_code_map          0000000000000000     <absolute>
 0000:00000000       __hybrid_code_map_count    0000000000000000     <absolute>
 0000:00000000       __x64_code_ranges_to_entry_points 0000000000000000     <absolute>
 0000:00000000       __x64_code_ranges_to_entry_points_count 0000000000000000     <absolute>
 0000:00000100       __guard_flags              0000000000000100     <absolute>
 0000:00000000       __ImageBase                0000000180000000     <linker-defined>
 0001:00000214       JNI_OnUnload               0000000180001214 f   NativeCrypto.obj
 0001:000002dc       Java_jdk_crypto_jniprovider_NativeCrypto_CBCFinalEncrypt 00000001800012dc f   NativeCrypto.obj
 0001:00000460       Java_jdk_crypto_jniprovider_NativeCrypto_CBCInit 0000000180001460 f   NativeCrypto.obj
 0001:000005c0       Java_jdk_crypto_jniprovider_NativeCrypto_CBCUpdate 00000001800015c0 f   NativeCrypto.obj
 0001:000006f0       Java_jdk_crypto_jniprovider_NativeCrypto_ChaCha20FinalDecrypt 00000001800016f0 f   NativeCrypto.obj
 0001:00000950       Java_jdk_crypto_jniprovider_NativeCrypto_ChaCha20FinalEncrypt 0000000180001950 f   NativeCrypto.obj
 0001:00000a1c       Java_jdk_crypto_jniprovider_NativeCrypto_ChaCha20Init 0000000180001a1c f   NativeCrypto.obj
 0001:00000c30       Java_jdk_crypto_jniprovider_NativeCrypto_ChaCha20Update 0000000180001c30 f   NativeCrypto.obj
 0001:00000e18       Java_jdk_crypto_jniprovider_NativeCrypto_CreateContext 0000000180001e18 f   NativeCrypto.obj
 0001:00000e38       Java_jdk_crypto_jniprovider_NativeCrypto_DestroyContext 0000000180001e38 f   NativeCrypto.obj
 0001:00000e58       Java_jdk_crypto_jniprovider_NativeCrypto_DigestComputeAndReset 0000000180001e58 f   NativeCrypto.obj
 0001:00000fc0       Java_jdk_crypto_jniprovider_NativeCrypto_DigestCreateContext 0000000180001fc0 f   NativeCrypto.obj
 0001:0000111c       Java_jdk_crypto_jniprovider_NativeCrypto_DigestDestroyContext 000000018000211c f   NativeCrypto.obj
 0001:00001168       Java_jdk_crypto_jniprovider_NativeCrypto_DigestReset 0000000180002168 f   NativeCrypto.obj
 0001:000011cc       Java_jdk_crypto_jniprovider_NativeCrypto_DigestUpdate 00000001800021cc f   NativeCrypto.obj
 0001:00001270       Java_jdk_crypto_jniprovider_NativeCrypto_ECCreatePrivateKey 0000000180002270 f   NativeCrypto.obj
 0001:00001318       Java_jdk_crypto_jniprovider_NativeCrypto_ECCreatePublicKey 0000000180002318 f   NativeCrypto.obj
 0001:0000143c       Java_jdk_crypto_jniprovider_NativeCrypto_ECDSASign 000000018000243c f   NativeCrypto.obj
 0001:00001578       Java_jdk_crypto_jniprovider_NativeCrypto_ECDSAVerify 0000000180002578 f   NativeCrypto.obj
 0001:000016c0       Java_jdk_crypto_jniprovider_NativeCrypto_ECDeriveKey 00000001800026c0 f   NativeCrypto.obj
 0001:00001768       Java_jdk_crypto_jniprovider_NativeCrypto_ECDestroyKey 0000000180002768 f   NativeCrypto.obj
 0001:00001788       Java_jdk_crypto_jniprovider_NativeCrypto_ECEncodeGF 0000000180002788 f   NativeCrypto.obj
 0001:00001b68       Java_jdk_crypto_jniprovider_NativeCrypto_ECGenerateKeyPair 0000000180002b68 f   NativeCrypto.obj
 0001:00001da8       Java_jdk_crypto_jniprovider_NativeCrypto_ECNativeGF2m 0000000180002da8 f   NativeCrypto.obj
 0001:00001db0       Java_jdk_crypto_jniprovider_NativeCrypto_GCMDecrypt 0000000180002db0 f   NativeCrypto.obj
 0001:00002110       Java_jdk_crypto_jniprovider_NativeCrypto_GCMEncrypt 0000000180003110 f   NativeCrypto.obj
 0001:00002458       Java_jdk_crypto_jniprovider_NativeCrypto_PBEDerive 0000000180003458 f   NativeCrypto.obj
 0001:000025f8       Java_jdk_crypto_jniprovider_NativeCrypto_PBKDF2Derive 00000001800035f8 f   NativeCrypto.obj
 0001:000027d0       Java_jdk_crypto_jniprovider_NativeCrypto_RSADP 00000001800037d0 f   NativeCrypto.obj
 0001:000029b0       Java_jdk_crypto_jniprovider_NativeCrypto_RSAEP 00000001800039b0 f   NativeCrypto.obj
 0001:00002a90       Java_jdk_crypto_jniprovider_NativeCrypto_XDHCreateKeys 0000000180003a90 f   NativeCrypto.obj
 0001:00002be4       Java_jdk_crypto_jniprovider_NativeCrypto_XDHGenerateSecret 0000000180003be4 f   NativeCrypto.obj
 0001:00002d90       Java_jdk_crypto_jniprovider_NativeCrypto_createRSAPrivateCrtKey 0000000180003d90 f   NativeCrypto.obj
 0001:00003488       Java_jdk_crypto_jniprovider_NativeCrypto_createRSAPublicKey 0000000180004488 f   NativeCrypto.obj
 0001:000035c4       Java_jdk_crypto_jniprovider_NativeCrypto_destroyRSAKey 00000001800045c4 f   NativeCrypto.obj
 0001:000035dc       Java_jdk_crypto_jniprovider_NativeCrypto_isMD5Available 00000001800045dc f   NativeCrypto.obj
 0001:000035e8       Java_jdk_crypto_jniprovider_NativeCrypto_isOpenSSLFIPS 00000001800045e8 f   NativeCrypto.obj
 0001:000035f0       Java_jdk_crypto_jniprovider_NativeCrypto_loadCrypto 00000001800045f0 f   NativeCrypto.obj
 0001:00004a40       OSSL102_RSA_set0_crt_params 0000000180005a40 f   NativeCrypto.obj
 0001:00004adc       OSSL102_RSA_set0_factors   0000000180005adc f   NativeCrypto.obj
 0001:00004b4c       OSSL102_RSA_set0_key       0000000180005b4c f   NativeCrypto.obj
 0001:00004bdc       __local_stdio_printf_options 0000000180005bdc f i NativeCrypto.obj
 0001:00004be4       __local_stdio_scanf_options 0000000180005be4 f i NativeCrypto.obj
 0001:00004bec       convertJavaBItoBN          0000000180005bec f   NativeCrypto.obj
 0001:00004eb0       fprintf                    0000000180005eb0 f i NativeCrypto.obj
 0001:00005280       printf                     0000000180006280 f i NativeCrypto.obj
 0001:000052d4       setECPublicCoordinates     00000001800062d4 f   NativeCrypto.obj
 0001:000052dc       setECPublicKey             00000001800062dc f   NativeCrypto.obj
 0001:000053d0       sscanf                     00000001800063d0 f i NativeCrypto.obj
 0001:000055a4       __GSHandlerCheck           00000001800065a4 f   MSVCRT:gshandler.obj
 0001:000055c4       __GSHandlerCheckCommon     00000001800065c4 f   MSVCRT:gshandler.obj
 0001:00005630       __security_check_cookie    0000000180006630 f   MSVCRT:amdsecgs.obj
 0001:00005970       _DllMainCRTStartup         0000000180006970 f   MSVCRT:dll_dllmain.obj
 0001:000059b0       __raise_securityfailure    00000001800069b0 f   MSVCRT:gs_report.obj
 0001:000059e4       __report_gsfailure         00000001800069e4 f   MSVCRT:gs_report.obj
 0001:00005b2c       __security_init_cookie     0000000180006b2c f   MSVCRT:gs_support.obj
 0001:00005bd8       DllMain                    0000000180006bd8 f   MSVCRT:dll_dllmain_stub.obj
 0001:00005bfc       ?__scrt_initialize_type_info@@YAXXZ 0000000180006bfc f   MSVCRT:tncleanup.obj
 0001:00005c0c       ?__scrt_uninitialize_type_info@@YAXXZ 0000000180006c0c f   MSVCRT:tncleanup.obj
 0001:00005c18       __scrt_initialize_default_local_stdio_options 0000000180006c18 f   MSVCRT:default_local_stdio_options.obj
 0001:00005c34       __scrt_acquire_startup_lock 0000000180006c34 f   MSVCRT:utility.obj
 0001:00005c70       __scrt_dllmain_after_initialize_c 0000000180006c70 f   MSVCRT:utility.obj
 0001:00005ca4       __scrt_dllmain_before_initialize_c 0000000180006ca4 f   MSVCRT:utility.obj
 0001:00005cbc       __scrt_dllmain_crt_thread_attach 0000000180006cbc f   MSVCRT:utility.obj
 0001:00005ce4       __scrt_dllmain_crt_thread_detach 0000000180006ce4 f   MSVCRT:utility.obj
 0001:00005cfc       __scrt_dllmain_exception_filter 0000000180006cfc f   MSVCRT:utility.obj
 0001:00005d5c       __scrt_dllmain_uninitialize_c 0000000180006d5c f   MSVCRT:utility.obj
 0001:00005d8c       __scrt_dllmain_uninitialize_critical 0000000180006d8c f   MSVCRT:utility.obj
 0001:00005da0       __scrt_initialize_crt      0000000180006da0 f   MSVCRT:utility.obj
 0001:00005dec       __scrt_initialize_onexit_tables 0000000180006dec f   MSVCRT:utility.obj
 0001:00005e78       __scrt_is_nonwritable_in_current_image 0000000180006e78 f   MSVCRT:utility.obj
 0001:00005f10       __scrt_release_startup_lock 0000000180006f10 f   MSVCRT:utility.obj
 0001:00005f34       __scrt_uninitialize_crt    0000000180006f34 f   MSVCRT:utility.obj
 0001:00005f60       __scrt_get_dyn_tls_init_callback 0000000180006f60 f   MSVCRT:dyn_tls_init.obj
 0001:00005f68       __crt_debugger_hook        0000000180006f68 f   MSVCRT:utility_desktop.obj
 0001:00005f70       __scrt_fastfail            0000000180006f70 f   MSVCRT:utility_desktop.obj
 0001:000060bc       _RTC_Initialize            00000001800070bc f   MSVCRT:initsect.obj
 0001:000060f8       _RTC_Terminate             00000001800070f8 f   MSVCRT:initsect.obj
 0001:00006134       _guard_check_icall_nop     0000000180007134 f i MSVCRT:guard_support.obj
 0001:00006138       __isa_available_init       0000000180007138 f   MSVCRT:cpu_disp.obj
 0001:000062e4       _get_startup_argv_mode     00000001800072e4 f   MSVCRT:argv_mode.obj
 0001:000062ec       __scrt_is_ucrt_dll_in_use  00000001800072ec f   MSVCRT:ucrt_detection.obj
 0001:00006300       memset                     0000000180007300 f   vcruntime:VCRUNTIME140.dll
 0001:00006306       __C_specific_handler       0000000180007306 f   vcruntime:VCRUNTIME140.dll
 0001:0000630c       __std_type_info_destroy_list 000000018000730c f   vcruntime:VCRUNTIME140.dll
 0001:00006312       strcat                     0000000180007312 f   ucrt:api-ms-win-crt-string-l1-1-0.dll
 0001:00006318       strcpy                     0000000180007318 f   ucrt:api-ms-win-crt-string-l1-1-0.dll
 0001:0000631e       strlen                     000000018000731e f   ucrt:api-ms-win-crt-string-l1-1-0.dll
 0001:00006324       _initterm                  0000000180007324 f   ucrt:api-ms-win-crt-runtime-l1-1-0.dll
 0001:0000632a       _initterm_e                000000018000732a f   ucrt:api-ms-win-crt-runtime-l1-1-0.dll
 0001:00006330       _seh_filter_dll            0000000180007330 f   ucrt:api-ms-win-crt-runtime-l1-1-0.dll
 0001:00006336       _configure_narrow_argv     0000000180007336 f   ucrt:api-ms-win-crt-runtime-l1-1-0.dll
 0001:0000633c       _initialize_narrow_environment 000000018000733c f   ucrt:api-ms-win-crt-runtime-l1-1-0.dll
 0001:00006342       _initialize_onexit_table   0000000180007342 f   ucrt:api-ms-win-crt-runtime-l1-1-0.dll
 0001:00006348       _execute_onexit_table      0000000180007348 f   ucrt:api-ms-win-crt-runtime-l1-1-0.dll
 0001:0000634e       _cexit                     000000018000734e f   ucrt:api-ms-win-crt-runtime-l1-1-0.dll
 0001:00006354       __acrt_initialize          0000000180007354 f   MSVCRT:ucrt_stubs.obj
 0001:00006354       __acrt_thread_attach       0000000180007354 f   MSVCRT:ucrt_stubs.obj
 0001:00006354       __acrt_thread_detach       0000000180007354 f   MSVCRT:ucrt_stubs.obj
 0001:00006354       __acrt_uninitialize        0000000180007354 f   MSVCRT:ucrt_stubs.obj
 0001:00006354       __acrt_uninitialize_critical 0000000180007354 f   MSVCRT:ucrt_stubs.obj
 0001:00006354       __scrt_stub_for_acrt_initialize 0000000180007354 f   MSVCRT:ucrt_stubs.obj
 0001:00006354       __scrt_stub_for_acrt_thread_attach 0000000180007354 f   MSVCRT:ucrt_stubs.obj
 0001:00006354       __scrt_stub_for_acrt_thread_detach 0000000180007354 f   MSVCRT:ucrt_stubs.obj
 0001:00006354       __scrt_stub_for_acrt_uninitialize 0000000180007354 f   MSVCRT:ucrt_stubs.obj
 0001:00006354       __scrt_stub_for_acrt_uninitialize_critical 0000000180007354 f   MSVCRT:ucrt_stubs.obj
 0001:00006354       __vcrt_initialize          0000000180007354 f   MSVCRT:ucrt_stubs.obj
 0001:00006354       __vcrt_thread_attach       0000000180007354 f   MSVCRT:ucrt_stubs.obj
 0001:00006354       __vcrt_thread_detach       0000000180007354 f   MSVCRT:ucrt_stubs.obj
 0001:00006354       __vcrt_uninitialize        0000000180007354 f   MSVCRT:ucrt_stubs.obj
 0001:00006354       __vcrt_uninitialize_critical 0000000180007354 f   MSVCRT:ucrt_stubs.obj
 0001:00006358       __scrt_stub_for_is_c_termination_complete 0000000180007358 f   MSVCRT:ucrt_stubs.obj
 0001:00006358       _is_c_termination_complete 0000000180007358 f   MSVCRT:ucrt_stubs.obj
 0001:0000635b       memcpy                     000000018000735b f   vcruntime:VCRUNTIME140.dll
 0001:00006380       _guard_dispatch_icall_nop  0000000180007380 f   MSVCRT:guard_dispatch.obj
 0001:000063a0       _guard_xfg_dispatch_icall_nop 00000001800073a0 f   MSVCRT:guard_xfg_dispatch.obj
 0002:00000000       __imp_CloseHandle          0000000180008000     kernel32:KERNEL32.dll
 0002:00000008       __imp_GetLastError         0000000180008008     kernel32:KERNEL32.dll
 0002:00000010       __imp_ReleaseMutex         0000000180008010     kernel32:KERNEL32.dll
 0002:00000018       __imp_WaitForSingleObject  0000000180008018     kernel32:KERNEL32.dll
 0002:00000020       __imp_CreateMutexA         0000000180008020     kernel32:KERNEL32.dll
 0002:00000028       __imp_FreeLibrary          0000000180008028     kernel32:KERNEL32.dll
 0002:00000030       __imp_GetModuleFileNameA   0000000180008030     kernel32:KERNEL32.dll
 0002:00000038       __imp_GetProcAddress       0000000180008038     kernel32:KERNEL32.dll
 0002:00000040       __imp_LoadLibraryA         0000000180008040     kernel32:KERNEL32.dll
 0002:00000048       __imp_LocalFree            0000000180008048     kernel32:KERNEL32.dll
 0002:00000050       __imp_FormatMessageA       0000000180008050     kernel32:KERNEL32.dll
 0002:00000058       __imp_RtlCaptureContext    0000000180008058     kernel32:KERNEL32.dll
 0002:00000060       __imp_RtlLookupFunctionEntry 0000000180008060     kernel32:KERNEL32.dll
 0002:00000068       __imp_RtlVirtualUnwind     0000000180008068     kernel32:KERNEL32.dll
 0002:00000070       __imp_UnhandledExceptionFilter 0000000180008070     kernel32:KERNEL32.dll
 0002:00000078       __imp_SetUnhandledExceptionFilter 0000000180008078     kernel32:KERNEL32.dll
 0002:00000080       __imp_GetCurrentProcess    0000000180008080     kernel32:KERNEL32.dll
 0002:00000088       __imp_TerminateProcess     0000000180008088     kernel32:KERNEL32.dll
 0002:00000090       __imp_IsProcessorFeaturePresent 0000000180008090     kernel32:KERNEL32.dll
 0002:00000098       __imp_QueryPerformanceCounter 0000000180008098     kernel32:KERNEL32.dll
 0002:000000a0       __imp_GetCurrentProcessId  00000001800080a0     kernel32:KERNEL32.dll
 0002:000000a8       __imp_GetCurrentThreadId   00000001800080a8     kernel32:KERNEL32.dll
 0002:000000b0       __imp_GetSystemTimeAsFileTime 00000001800080b0     kernel32:KERNEL32.dll
 0002:000000b8       __imp_DisableThreadLibraryCalls 00000001800080b8     kernel32:KERNEL32.dll
 0002:000000c0       __imp_InitializeSListHead  00000001800080c0     kernel32:KERNEL32.dll
 0002:000000c8       __imp_IsDebuggerPresent    00000001800080c8     kernel32:KERNEL32.dll
 0002:000000d0       \177KERNEL32_NULL_THUNK_DATA 00000001800080d0     kernel32:KERNEL32.dll
 0002:000000d8       __imp_memset               00000001800080d8     vcruntime:VCRUNTIME140.dll
 0002:000000e0       __imp___C_specific_handler 00000001800080e0     vcruntime:VCRUNTIME140.dll
 0002:000000e8       __imp___std_type_info_destroy_list 00000001800080e8     vcruntime:VCRUNTIME140.dll
 0002:000000f0       __imp_memcpy               00000001800080f0     vcruntime:VCRUNTIME140.dll
 0002:000000f8       \177VCRUNTIME140_NULL_THUNK_DATA 00000001800080f8     vcruntime:VCRUNTIME140.dll
 0002:00000100       __imp_malloc               0000000180008100     ucrt:api-ms-win-crt-heap-l1-1-0.dll
 0002:00000108       __imp_free                 0000000180008108     ucrt:api-ms-win-crt-heap-l1-1-0.dll
 0002:00000110       \177api-ms-win-crt-heap-l1-1-0_NULL_THUNK_DATA 0000000180008110     ucrt:api-ms-win-crt-heap-l1-1-0.dll
 0002:00000118       __imp__cexit               0000000180008118     ucrt:api-ms-win-crt-runtime-l1-1-0.dll
 0002:00000120       __imp__execute_onexit_table 0000000180008120     ucrt:api-ms-win-crt-runtime-l1-1-0.dll
 0002:00000128       __imp__configure_narrow_argv 0000000180008128     ucrt:api-ms-win-crt-runtime-l1-1-0.dll
 0002:00000130       __imp__initterm            0000000180008130     ucrt:api-ms-win-crt-runtime-l1-1-0.dll
 0002:00000138       __imp__initterm_e          0000000180008138     ucrt:api-ms-win-crt-runtime-l1-1-0.dll
 0002:00000140       __imp__initialize_onexit_table 0000000180008140     ucrt:api-ms-win-crt-runtime-l1-1-0.dll
 0002:00000148       __imp__seh_filter_dll      0000000180008148     ucrt:api-ms-win-crt-runtime-l1-1-0.dll
 0002:00000150       __imp__initialize_narrow_environment 0000000180008150     ucrt:api-ms-win-crt-runtime-l1-1-0.dll
 0002:00000158       \177api-ms-win-crt-runtime-l1-1-0_NULL_THUNK_DATA 0000000180008158     ucrt:api-ms-win-crt-runtime-l1-1-0.dll
 0002:00000160       __imp___stdio_common_vfprintf 0000000180008160     ucrt:api-ms-win-crt-stdio-l1-1-0.dll
 0002:00000168       __imp_fflush               0000000180008168     ucrt:api-ms-win-crt-stdio-l1-1-0.dll
 0002:00000170       __imp___stdio_common_vsscanf 0000000180008170     ucrt:api-ms-win-crt-stdio-l1-1-0.dll
 0002:00000178       __imp___acrt_iob_func      0000000180008178     ucrt:api-ms-win-crt-stdio-l1-1-0.dll
 0002:00000180       \177api-ms-win-crt-stdio-l1-1-0_NULL_THUNK_DATA 0000000180008180     ucrt:api-ms-win-crt-stdio-l1-1-0.dll
 0002:00000188       __imp_strlen               0000000180008188     ucrt:api-ms-win-crt-string-l1-1-0.dll
 0002:00000190       __imp_isalpha              0000000180008190     ucrt:api-ms-win-crt-string-l1-1-0.dll
 0002:00000198       __imp_strcpy               0000000180008198     ucrt:api-ms-win-crt-string-l1-1-0.dll
 0002:000001a0       __imp_strcat               00000001800081a0     ucrt:api-ms-win-crt-string-l1-1-0.dll
 0002:000001a8       __imp_tolower              00000001800081a8     ucrt:api-ms-win-crt-string-l1-1-0.dll
 0002:000001b0       \177api-ms-win-crt-string-l1-1-0_NULL_THUNK_DATA 00000001800081b0     ucrt:api-ms-win-crt-string-l1-1-0.dll
 0002:000001b8       __guard_check_icall_fptr   00000001800081b8     MSVCRT:guard_support.obj
 0002:000001c0       __guard_xfg_check_icall_fptr 00000001800081c0     MSVCRT:guard_support.obj
 0002:000001c8       __guard_dispatch_icall_fptr 00000001800081c8     MSVCRT:guard_support.obj
 0002:000001d0       __guard_xfg_dispatch_icall_fptr 00000001800081d0     MSVCRT:guard_support.obj
 0002:000001d8       __guard_xfg_table_dispatch_icall_fptr 00000001800081d8     MSVCRT:guard_support.obj
 0002:000001e0       __castguard_check_failure_os_handled_fptr 00000001800081e0     MSVCRT:guard_support.obj
 0002:000001e8       __guard_memcpy_fptr        00000001800081e8     vcruntime:softmemtag.obj
 0002:000001f0       __xc_a                     00000001800081f0     MSVCRT:initializers.obj
 0002:000001f8       __xc_z                     00000001800081f8     MSVCRT:initializers.obj
 0002:00000200       __xi_a                     0000000180008200     MSVCRT:initializers.obj
 0002:00000208       __xi_z                     0000000180008208     MSVCRT:initializers.obj
 0002:00000210       __xp_a                     0000000180008210     MSVCRT:initializers.obj
 0002:00000218       __xp_z                     0000000180008218     MSVCRT:initializers.obj
 0002:00000220       __xt_a                     0000000180008220     MSVCRT:initializers.obj
 0002:00000228       __xt_z                     0000000180008228     MSVCRT:initializers.obj
 0002:00000268       ??_C@_0BL@JFKAOCIF@An?5OpenSSL?5error?5occurred?6@ 0000000180008268     NativeCrypto.obj
 0002:00000284       ??_C@_03OFAPEBGM@?$CFs?6@  0000000180008284     NativeCrypto.obj
 0002:00000288       ??_C@_0BG@MBINOMKO@OpenSSL?5?$CFld?4?$CFld?4?$CFld?$CFc@ 0000000180008288     NativeCrypto.obj
 0002:000002a0       ??_C@_0BO@FCDFIFHK@OpenSSL?5was?5loaded?5from?5?9?5?$CFs?6@ 00000001800082a0     NativeCrypto.obj
 0002:000002c0       ??_C@_0BA@HPMBCNAB@OpenSSL_version@ 00000001800082c0     NativeCrypto.obj
 0002:000002d0       ??_C@_0P@PIHLHJGN@SSLeay_version@ 00000001800082d0     NativeCrypto.obj
 0002:000002e0       ??_C@_0FH@BAFCINAE@Error?5loading?5OpenSSL?3?5Error?5fi@ 00000001800082e0     NativeCrypto.obj
 0002:00000338       ??_C@_0DP@JGPDADLC@Error?5loading?5OpenSSL?3?5Incompat@ 0000000180008338     NativeCrypto.obj
 0002:00000378       ??_C@_0CH@LOBKHAIN@EVP_default_properties_is_fips_@ 0000000180008378     NativeCrypto.obj
 0002:000003a0       ??_C@_09BCJAEHEL@FIPS_mode@ 00000001800083a0     NativeCrypto.obj
 0002:000003b0       ??_C@_07KJFPOMFC@?$CFs?3?5?$CFs?6@ 00000001800083b0     NativeCrypto.obj
 0002:000003b8       ??_C@_0BB@CMEKANCH@?$CIunknown?5reason?$CJ@ 00000001800083b8     NativeCrypto.obj
 0002:000003d0       ??_C@_0BN@PCLDIFCP@Failed?5to?5load?5?$CFs?5due?5to?5?$CFs?6@ 00000001800083d0     NativeCrypto.obj
 0002:000003f0       ??_C@_0BE@ENBECKJM@libcrypto?93?9x64?4dll@ 00000001800083f0     NativeCrypto.obj
 0002:00000408       ??_C@_0BG@EJIPPMGK@libcrypto?91_1?9x64?4dll@ 0000000180008408     NativeCrypto.obj
 0002:00000420       ??_C@_0N@IEEBINGH@libeay32?4dll@ 0000000180008420     NativeCrypto.obj
 0002:00000430       ??_C@_0DI@PFJKEFNN@Skipping?5trying?5to?5load?5a?5libra@ 0000000180008430     NativeCrypto.obj
 0002:00000468       ??_C@_0CG@LKMEGFEO@?7Failed?5to?5allocate?5memory?5for?5@ 0000000180008468     NativeCrypto.obj
 0002:00000490       ??_C@_0DG@BHEPPKLO@Attempting?5to?5load?5library?5bund@ 0000000180008490     NativeCrypto.obj
 0002:000004c8       ??_C@_0BJ@IJGPDENH@?7Attempting?5to?5load?3?5?$CFs?6@ 00000001800084c8     NativeCrypto.obj
 0002:000004e8       ??_C@_0BJ@BOLPKGOH@?7?7Loaded?5OpenSSL?5version@ 00000001800084e8     NativeCrypto.obj
 0002:00000508       ??_C@_0CI@GFBPIMLI@Attempting?5to?5load?5libname?5from@ 0000000180008508     NativeCrypto.obj
 0002:00000530       ??_C@_0BI@NNDBGBPB@?7Loaded?5OpenSSL?5version@ 0000000180008530     NativeCrypto.obj
 0002:00000548       ??_C@_00CNPNBAHC@@         0000000180008548     NativeCrypto.obj
 0002:00000550       ??_C@_0CN@KCODGBDO@Failed?5to?5get?5jdk?4native?4openss@ 0000000180008550     NativeCrypto.obj
 0002:00000580       ??_C@_0DB@KNFOOGBB@The?5jdk?4native?4openssl?4lib?5prop@ 0000000180008580     NativeCrypto.obj
 0002:000005c0       ??_C@_0EC@CELBJHCF@OpenSSL?5library?5specified?5in?5jd@ 00000001800085c0     NativeCrypto.obj
 0002:00000608       ??_C@_0CA@LGHBIFJG@Failed?5to?5get?5java?4home?5value?4?6@ 0000000180008608     NativeCrypto.obj
 0002:00000628       ??_C@_0CH@GMNJBKEN@FAILED?5TO?5LOAD?5OPENSSL?5CRYPTO?5L@ 0000000180008628     NativeCrypto.obj
 0002:00000650       ??_C@_0CI@NJCDBAGM@Version?5of?5OpenSSL?5library?5that@ 0000000180008650     NativeCrypto.obj
 0002:00000678       ??_C@_0BD@KCMFIFPA@ERR_error_string_n@ 0000000180008678     NativeCrypto.obj
 0002:00000690       ??_C@_0BB@GICHBNCI@ERR_error_string@ 0000000180008690     NativeCrypto.obj
 0002:000006a8       ??_C@_0O@CFFJHPAB@ERR_get_error@ 00000001800086a8     NativeCrypto.obj
 0002:000006b8       ??_C@_0BB@COGJFOLI@CRYPTO_num_locks@ 00000001800086b8     NativeCrypto.obj
 0002:000006d0       ??_C@_0BM@BPNHJJIG@CRYPTO_THREADID_set_numeric@ 00000001800086d0     NativeCrypto.obj
 0002:000006f0       ??_C@_0O@JHFEPHEL@CRYPTO_malloc@ 00000001800086f0     NativeCrypto.obj
 0002:00000700       ??_C@_0M@MLHDOKNM@CRYPTO_free@ 0000000180008700     NativeCrypto.obj
 0002:00000710       ??_C@_0BN@KPFPHOHH@CRYPTO_THREADID_set_callback@ 0000000180008710     NativeCrypto.obj
 0002:00000730       ??_C@_0BM@IOPFJNF@CRYPTO_set_locking_callback@ 0000000180008730     NativeCrypto.obj
 0002:00000750       ??_C@_07CJMLOOOL@EVP_md5@  0000000180008750     NativeCrypto.obj
 0002:00000758       ??_C@_08PBPOHJL@EVP_sha1@  0000000180008758     NativeCrypto.obj
 0002:00000768       ??_C@_0L@BFNCDCPF@EVP_sha256@ 0000000180008768     NativeCrypto.obj
 0002:00000778       ??_C@_0L@CCKLEGPC@EVP_sha224@ 0000000180008778     NativeCrypto.obj
 0002:00000788       ??_C@_0L@JHIAKEEB@EVP_sha384@ 0000000180008788     NativeCrypto.obj
 0002:00000798       ??_C@_0L@OLGAGHJE@EVP_sha512@ 0000000180008798     NativeCrypto.obj
 0002:000007a8       ??_C@_0P@FBDLFBDI@EVP_sha512_224@ 00000001800087a8     NativeCrypto.obj
 0002:000007b8       ??_C@_0P@GGECCFDP@EVP_sha512_256@ 00000001800087b8     NativeCrypto.obj
 0002:000007c8       ??_C@_0P@LBBHIKLM@EVP_MD_CTX_new@ 00000001800087c8     NativeCrypto.obj
 0002:000007d8       ??_C@_0BB@LLCENKBD@EVP_MD_CTX_reset@ 00000001800087d8     NativeCrypto.obj
 0002:000007f0       ??_C@_0BA@DIPACEDG@EVP_MD_CTX_free@ 00000001800087f0     NativeCrypto.obj
 0002:00000800       ??_C@_0BC@CDDHKKMK@EVP_MD_CTX_create@ 0000000180008800     NativeCrypto.obj
 0002:00000818       ??_C@_0BD@EAMOJGOK@EVP_MD_CTX_cleanup@ 0000000180008818     NativeCrypto.obj
 0002:00000830       ??_C@_0BD@HIKAFGJM@EVP_MD_CTX_destroy@ 0000000180008830     NativeCrypto.obj
 0002:00000848       ??_C@_0BC@NBJFCNLO@EVP_DigestInit_ex@ 0000000180008848     NativeCrypto.obj
 0002:00000860       ??_C@_0BD@OOMFHFKA@EVP_MD_CTX_copy_ex@ 0000000180008860     NativeCrypto.obj
 0002:00000878       ??_C@_0BB@ECHJOJOG@EVP_DigestUpdate@ 0000000180008878     NativeCrypto.obj
 0002:00000890       ??_C@_0BD@OFMHHJIG@EVP_DigestFinal_ex@ 0000000180008890     NativeCrypto.obj
 0002:000008a8       ??_C@_0BD@KDJHKKHN@EVP_CIPHER_CTX_new@ 00000001800088a8     NativeCrypto.obj
 0002:000008c0       ??_C@_0BE@NEIBFGDA@EVP_CIPHER_CTX_free@ 00000001800088c0     NativeCrypto.obj
 0002:000008d8       ??_C@_0BA@MIPBGJPL@EVP_aes_128_cbc@ 00000001800088d8     NativeCrypto.obj
 0002:000008e8       ??_C@_0BA@GLGNBOGH@EVP_aes_192_cbc@ 00000001800088e8     NativeCrypto.obj
 0002:000008f8       ??_C@_0BA@LJNDDBOG@EVP_aes_256_cbc@ 00000001800088f8     NativeCrypto.obj
 0002:00000908       ??_C@_0BC@FOOGEGCP@EVP_CipherInit_ex@ 0000000180008908     NativeCrypto.obj
 0002:00000920       ??_C@_0BL@GHJMPLKJ@EVP_CIPHER_CTX_set_padding@ 0000000180008920     NativeCrypto.obj
 0002:00000940       ??_C@_0BB@FEIMIHDK@EVP_CipherUpdate@ 0000000180008940     NativeCrypto.obj
 0002:00000958       ??_C@_0BD@GCEAKJDP@EVP_CipherFinal_ex@ 0000000180008958     NativeCrypto.obj
 0002:00000970       ??_C@_0BA@NINCLJBF@EVP_aes_128_gcm@ 0000000180008970     NativeCrypto.obj
 0002:00000980       ??_C@_0BA@HLEOMOIJ@EVP_aes_192_gcm@ 0000000180008980     NativeCrypto.obj
 0002:00000990       ??_C@_0BA@KJPAOBAI@EVP_aes_256_gcm@ 0000000180008990     NativeCrypto.obj
 0002:000009a0       ??_C@_0BE@PBKBIICA@EVP_CIPHER_CTX_ctrl@ 00000001800089a0     NativeCrypto.obj
 0002:000009b8       ??_C@_0BD@NJDNKKJM@EVP_DecryptInit_ex@ 00000001800089b8     NativeCrypto.obj
 0002:000009d0       ??_C@_0BC@IHMDOGKL@EVP_DecryptUpdate@ 00000001800089d0     NativeCrypto.obj
 0002:000009e8       ??_C@_0BB@PDIJBBLN@EVP_DecryptFinal@ 00000001800089e8     NativeCrypto.obj
 0002:00000a00       ??_C@_0N@KEPOPDOF@EVP_chacha20@ 0000000180008a00     NativeCrypto.obj
 0002:00000a10       ??_C@_0BG@JOEAPCLB@EVP_chacha20_poly1305@ 0000000180008a10     NativeCrypto.obj
 0002:00000a28       ??_C@_07BEDPMABO@RSA_new@  0000000180008a28     NativeCrypto.obj
 0002:00000a30       ??_C@_0N@CGJMOJGH@RSA_set0_key@ 0000000180008a30     NativeCrypto.obj
 0002:00000a40       ??_C@_0BB@POEMEDBA@RSA_set0_factors@ 0000000180008a40     NativeCrypto.obj
 0002:00000a58       ??_C@_0BE@IHFICCGA@RSA_set0_crt_params@ 0000000180008a58     NativeCrypto.obj
 0002:00000a70       ??_C@_08INMOLI@RSA_free@   0000000180008a70     NativeCrypto.obj
 0002:00000a80       ??_C@_0BD@PDPPPPCN@RSA_public_decrypt@ 0000000180008a80     NativeCrypto.obj
 0002:00000a98       ??_C@_0BE@GMELDCOG@RSA_private_decrypt@ 0000000180008a98     NativeCrypto.obj
 0002:00000aac       ??_C@_06MLINBBBN@BN_new@   0000000180008aac     NativeCrypto.obj
 0002:00000ab8       ??_C@_09ODLDNKNE@BN_bin2bn@ 0000000180008ab8     NativeCrypto.obj
 0002:00000ac8       ??_C@_0BA@NODPKDEN@BN_set_negative@ 0000000180008ac8     NativeCrypto.obj
 0002:00000ad8       ??_C@_07JJFLCNND@BN_free@  0000000180008ad8     NativeCrypto.obj
 0002:00000ae0       ??_C@_09MEANCIOF@BN_bn2bin@ 0000000180008ae0     NativeCrypto.obj
 0002:00000af0       ??_C@_0M@BMNNLAL@BN_num_bits@ 0000000180008af0     NativeCrypto.obj
 0002:00000b00       ??_C@_0BE@MFFKFHAB@EC_KEY_generate_key@ 0000000180008b00     NativeCrypto.obj
 0002:00000b18       ??_C@_0M@NMKCGAJN@EC_KEY_free@ 0000000180008b18     NativeCrypto.obj
 0002:00000b28       ??_C@_0BB@IOKCFGPF@ECDH_compute_key@ 0000000180008b28     NativeCrypto.obj
 0002:00000b40       ??_C@_0BH@OFCAHLIM@EC_KEY_get0_public_key@ 0000000180008b40     NativeCrypto.obj
 0002:00000b58       ??_C@_0BI@IHBMKFAL@EC_KEY_get0_private_key@ 0000000180008b58     NativeCrypto.obj
 0002:00000b70       ??_C@_0L@ONJMCKDA@EC_KEY_new@ 0000000180008b70     NativeCrypto.obj
 0002:00000b80       ??_C@_0CJ@PKPNGFF@EC_KEY_set_public_key_affine_co@ 0000000180008b80     NativeCrypto.obj
 0002:00000bb0       ??_C@_0BH@ELJHICGP@EC_KEY_set_private_key@ 0000000180008bb0     NativeCrypto.obj
 0002:00000bc8       ??_C@_0L@OIEJOLGJ@BN_CTX_new@ 0000000180008bc8     NativeCrypto.obj
 0002:00000bd8       ??_C@_0BH@LMGLLNHD@EC_GROUP_new_curve_GFp@ 0000000180008bd8     NativeCrypto.obj
 0002:00000bf0       ??_C@_0BI@GKPNAHHP@EC_GROUP_new_curve_GF2m@ 0000000180008bf0     NativeCrypto.obj
 0002:00000c08       ??_C@_0BB@NIEGABFH@EC_KEY_set_group@ 0000000180008c08     NativeCrypto.obj
 0002:00000c20       ??_C@_0N@LOIMDOGK@EC_POINT_new@ 0000000180008c20     NativeCrypto.obj
 0002:00000c30       ??_C@_0BH@CFECBPOO@EC_GROUP_set_generator@ 0000000180008c30     NativeCrypto.obj
 0002:00000c48       ??_C@_0BC@KEIEKAMA@EC_KEY_get0_group@ 0000000180008c48     NativeCrypto.obj
 0002:00000c60       ??_C@_0O@FHEPMIGD@EC_POINT_free@ 0000000180008c60     NativeCrypto.obj
 0002:00000c70       ??_C@_0O@KEFGGDJH@EC_GROUP_free@ 0000000180008c70     NativeCrypto.obj
 0002:00000c80       ??_C@_0M@MOBAFMAM@BN_CTX_free@ 0000000180008c80     NativeCrypto.obj
 0002:00000c90       ??_C@_0BG@GCHAIKDI@EC_KEY_set_public_key@ 0000000180008c90     NativeCrypto.obj
 0002:00000ca8       ??_C@_0BB@NNGADNNL@EC_KEY_check_key@ 0000000180008ca8     NativeCrypto.obj
 0002:00000cc0       ??_C@_0CA@GKCLEFHF@EC_POINT_set_affine_coordinates@ 0000000180008cc0     NativeCrypto.obj
 0002:00000ce0       ??_C@_0CA@GLAFGCKK@EC_POINT_get_affine_coordinates@ 0000000180008ce0     NativeCrypto.obj
 0002:00000d00       ??_C@_0CE@BGAPNKLA@EC_POINT_set_affine_coordinates@ 0000000180008d00     NativeCrypto.obj
 0002:00000d28       ??_C@_0CF@GIDKPABC@EC_POINT_set_affine_coordinates@ 0000000180008d28     NativeCrypto.obj
 0002:00000d50       ??_C@_0CE@CJDKBKKA@EC_POINT_get_affine_coordinates@ 0000000180008d50     NativeCrypto.obj
 0002:00000d78       ??_C@_0CF@HFLCNFLG@EC_POINT_get_affine_coordinates@ 0000000180008d78     NativeCrypto.obj
 0002:00000da0       ??_C@_0BB@CDDFLDAE@EVP_PKEY_CTX_new@ 0000000180008da0     NativeCrypto.obj
 0002:00000db8       ??_C@_0BE@ELKLNAFP@EVP_PKEY_CTX_new_id@ 0000000180008db8     NativeCrypto.obj
 0002:00000dd0       ??_C@_0BF@HNJPEBIC@EVP_PKEY_keygen_init@ 0000000180008dd0     NativeCrypto.obj
 0002:00000de8       ??_C@_0BA@DHFOBMEL@EVP_PKEY_keygen@ 0000000180008de8     NativeCrypto.obj
 0002:00000df8       ??_C@_0BC@PNNIDNLB@EVP_PKEY_CTX_free@ 0000000180008df8     NativeCrypto.obj
 0002:00000e10       ??_C@_0BN@HEFFNPAD@EVP_PKEY_get_raw_private_key@ 0000000180008e10     NativeCrypto.obj
 0002:00000e30       ??_C@_0BM@BFCLDLJO@EVP_PKEY_get_raw_public_key@ 0000000180008e30     NativeCrypto.obj
 0002:00000e50       ??_C@_0BN@GGGPOPJF@EVP_PKEY_new_raw_private_key@ 0000000180008e50     NativeCrypto.obj
 0002:00000e70       ??_C@_0BM@JIPCPNMH@EVP_PKEY_new_raw_public_key@ 0000000180008e70     NativeCrypto.obj
 0002:00000e90       ??_C@_0BF@MPBKJMKE@EVP_PKEY_derive_init@ 0000000180008e90     NativeCrypto.obj
 0002:00000ea8       ??_C@_0BJ@CECPMDDP@EVP_PKEY_derive_set_peer@ 0000000180008ea8     NativeCrypto.obj
 0002:00000ec8       ??_C@_0BA@KLINOOGC@EVP_PKEY_derive@ 0000000180008ec8     NativeCrypto.obj
 0002:00000ed8       ??_C@_0O@NLOFDJGI@EVP_PKEY_free@ 0000000180008ed8     NativeCrypto.obj
 0002:00000ee8       ??_C@_0O@HPIOKGCH@ECDSA_do_sign@ 0000000180008ee8     NativeCrypto.obj
 0002:00000ef8       ??_C@_0BA@EHPKHBIM@ECDSA_do_verify@ 0000000180008ef8     NativeCrypto.obj
 0002:00000f08       ??_C@_0O@LCAMPHNJ@ECDSA_SIG_new@ 0000000180008f08     NativeCrypto.obj
 0002:00000f18       ??_C@_0P@FCLKKJM@ECDSA_SIG_free@ 0000000180008f18     NativeCrypto.obj
 0002:00000f28       ??_C@_0BB@IIOJIAAH@ECDSA_SIG_get0_r@ 0000000180008f28     NativeCrypto.obj
 0002:00000f40       ??_C@_0BB@JBPCLBEG@ECDSA_SIG_get0_s@ 0000000180008f40     NativeCrypto.obj
 0002:00000f58       ??_C@_0P@LKMNLNBO@ECDSA_SIG_set0@ 0000000180008f58     NativeCrypto.obj
 0002:00000f68       ??_C@_0BD@DMMKPAAN@PKCS12_key_gen_uni@ 0000000180008f68     NativeCrypto.obj
 0002:00000f80       ??_C@_0BC@KMIHJAOO@PKCS5_PBKDF2_HMAC@ 0000000180008f80     NativeCrypto.obj
 0002:00000fa0       ??_C@_0EI@MPDAOHNE@Error?5loading?5OpenSSL?3?5One?5or?5m@ 0000000180008fa0     NativeCrypto.obj
 0002:00000fe8       ??_C@_0DG@CJHOCNOH@Error?5loading?5OpenSSL?3?5Thread?5s@ 0000000180008fe8     NativeCrypto.obj
 0002:00001020       ??_C@_0CG@HPEIDEDC@OpenSSL?5library?5loaded?5successf@ 0000000180009020     NativeCrypto.obj
 0002:00001048       ??_C@_0BH@KCAMECBI@CreateMutex?5error?3?5?$CFd?6@ 0000000180009048     NativeCrypto.obj
 0002:00001060       ??_C@_0BH@FPGCIENB@CloseHandle?5error?3?5?$CFd?6@ 0000000180009060     NativeCrypto.obj
 0002:00001078       ??_C@_0BP@OBCPLEDE@WaitForSingleObject?5error?3?5?$CFd?6@ 0000000180009078     NativeCrypto.obj
 0002:00001098       ??_C@_0BI@DELFCGJD@ReleaseMutex?5error?3?5?$CFd?6@ 0000000180009098     NativeCrypto.obj
 0002:000010b0       ??_C@_0BJ@LFBOMBKK@destoryResult?5error?3?5?$CFd?6@ 00000001800090b0     NativeCrypto.obj
 0002:000010d0       ??_C@_0CG@LFHDDGAP@Failed?5to?5create?5an?5ECDSA?5Signa@ 00000001800090d0     NativeCrypto.obj
 0002:000010f8       _pDefaultRawDllMain        00000001800090f8     MSVCRT:dll_dllmain.obj
 0002:000010f8       _pRawDllMain               00000001800090f8     MSVCRT:dll_dllmain.obj
 0002:00001110       __xmm@ffffffffffffffffffffffffffffffff 0000000180009110     MSVCRT:utility.obj
 0002:00001120       _load_config_used          0000000180009120     MSVCRT:loadcfg.obj
 0002:00001300       __volatile_metadata        0000000180009300     <linker-defined>
 0002:00001620       __rtc_iaa                  0000000180009620     MSVCRT:initsect.obj
 0002:00001628       __rtc_izz                  0000000180009628     MSVCRT:initsect.obj
 0002:00001630       __rtc_taa                  0000000180009630     MSVCRT:initsect.obj
 0002:00001638       __rtc_tzz                  0000000180009638     MSVCRT:initsect.obj
 0002:00002470       __IMPORT_DESCRIPTOR_KERNEL32 000000018000a470     kernel32:KERNEL32.dll
 0002:00002484       __IMPORT_DESCRIPTOR_VCRUNTIME140 000000018000a484     vcruntime:VCRUNTIME140.dll
 0002:00002498       __IMPORT_DESCRIPTOR_api-ms-win-crt-string-l1-1-0 000000018000a498     ucrt:api-ms-win-crt-string-l1-1-0.dll
 0002:000024ac       __IMPORT_DESCRIPTOR_api-ms-win-crt-stdio-l1-1-0 000000018000a4ac     ucrt:api-ms-win-crt-stdio-l1-1-0.dll
 0002:000024c0       __IMPORT_DESCRIPTOR_api-ms-win-crt-heap-l1-1-0 000000018000a4c0     ucrt:api-ms-win-crt-heap-l1-1-0.dll
 0002:000024d4       __IMPORT_DESCRIPTOR_api-ms-win-crt-runtime-l1-1-0 000000018000a4d4     ucrt:api-ms-win-crt-runtime-l1-1-0.dll
 0002:000024e8       __NULL_IMPORT_DESCRIPTOR   000000018000a4e8     kernel32:KERNEL32.dll
 0003:00000000       __security_cookie          000000018000b000     MSVCRT:gs_cookie.obj
 0003:00000008       __security_cookie_complement 000000018000b008     MSVCRT:gs_cookie.obj
 0003:00000010       __scrt_native_dllmain_reason 000000018000b010     MSVCRT:utility.obj
 0003:00000018       __isa_available            000000018000b018     MSVCRT:cpu_disp.obj
 0003:0000001c       __isa_enabled              000000018000b01c     MSVCRT:cpu_disp.obj
 0003:00000020       __memset_fast_string_threshold 000000018000b020     MSVCRT:cpu_disp.obj
 0003:00000028       __memset_nt_threshold      000000018000b028     MSVCRT:cpu_disp.obj
 0003:00000030       __scrt_ucrt_dll_is_in_use  000000018000b030     MSVCRT:ucrt_stubs.obj
 0003:00000040       first_time_gcm             000000018000b040     NativeCrypto.obj
 0003:00000600       ?__type_info_root_node@@3U__type_info_node@@A 000000018000b600     MSVCRT:tncleanup.obj
 0003:00000610       __scrt_current_native_startup_state 000000018000b610     MSVCRT:utility.obj
 0003:00000618       __scrt_native_startup_lock 000000018000b618     MSVCRT:utility.obj
 0003:00000658       __scrt_debugger_hook_flag  000000018000b658     MSVCRT:utility_desktop.obj
 0003:0000065c       __favor                    000000018000b65c     MSVCRT:cpu_disp.obj
 0003:00000660       ?_OptionsStorage@?1??__local_stdio_scanf_options@@9@9 000000018000b660     <common>
 0003:00000668       ?_OptionsStorage@?1??__local_stdio_printf_options@@9@9 000000018000b668     <common>
 0003:00000670       OSSL_PKCS5_PBKDF2_HMAC     000000018000b670     <common>
 0003:00000678       OSSL_PKCS12_key_gen        000000018000b678     <common>
 0003:00000680       OSSL_EVP_PKEY_free         000000018000b680     <common>
 0003:00000688       OSSL_EVP_PKEY_derive       000000018000b688     <common>
 0003:00000690       OSSL_EVP_PKEY_derive_set_peer 000000018000b690     <common>
 0003:00000698       OSSL_EVP_PKEY_derive_init  000000018000b698     <common>
 0003:000006a0       OSSL_EVP_PKEY_new_raw_public_key 000000018000b6a0     <common>
 0003:000006a8       OSSL_EVP_PKEY_new_raw_private_key 000000018000b6a8     <common>
 0003:000006b0       OSSL_EVP_PKEY_get_raw_public_key 000000018000b6b0     <common>
 0003:000006b8       OSSL_EVP_PKEY_get_raw_private_key 000000018000b6b8     <common>
 0003:000006c0       OSSL_EVP_PKEY_CTX_free     000000018000b6c0     <common>
 0003:000006c8       OSSL_EVP_PKEY_keygen       000000018000b6c8     <common>
 0003:000006d0       OSSL_EVP_PKEY_keygen_init  000000018000b6d0     <common>
 0003:000006d8       OSSL_EVP_PKEY_CTX_new_id   000000018000b6d8     <common>
 0003:000006e0       OSSL_EVP_PKEY_CTX_new      000000018000b6e0     <common>
 0003:000006e8       OSSL_ECDSA_SIG_set0        000000018000b6e8     <common>
 0003:000006f0       OSSL_ECDSA_SIG_get0_s      000000018000b6f0     <common>
 0003:000006f8       OSSL_ECDSA_SIG_get0_r      000000018000b6f8     <common>
 0003:00000700       OSSL_ECDSA_SIG_free        000000018000b700     <common>
 0003:00000708       OSSL_ECDSA_SIG_new         000000018000b708     <common>
 0003:00000710       OSSL_ECDSA_do_verify       000000018000b710     <common>
 0003:00000718       OSSL_ECDSA_do_sign         000000018000b718     <common>
 0003:00000720       OSSL_EC_KEY_get0_private_key 000000018000b720     <common>
 0003:00000728       EC_set_public_key          000000018000b728     <common>
 0003:00000730       OSSL_EC_KEY_check_key      000000018000b730     <common>
 0003:00000738       OSSL_EC_KEY_set_public_key 000000018000b738     <common>
 0003:00000740       OSSL_BN_CTX_free           000000018000b740     <common>
 0003:00000748       OSSL_EC_GROUP_free         000000018000b748     <common>
 0003:00000750       OSSL_EC_POINT_free         000000018000b750     <common>
 0003:00000758       OSSL_EC_KEY_get0_group     000000018000b758     <common>
 0003:00000760       OSSL_EC_GROUP_set_generator 000000018000b760     <common>
 0003:00000768       OSSL_EC_POINT_get_affine_coordinates_GF2m 000000018000b768     <common>
 0003:00000770       OSSL_EC_POINT_get_affine_coordinates_GFp 000000018000b770     <common>
 0003:00000778       OSSL_EC_POINT_set_affine_coordinates_GF2m 000000018000b778     <common>
 0003:00000780       OSSL_EC_POINT_set_affine_coordinates_GFp 000000018000b780     <common>
 0003:00000788       OSSL_EC_POINT_new          000000018000b788     <common>
 0003:00000790       OSSL_EC_KEY_set_group      000000018000b790     <common>
 0003:00000798       OSSL_EC_GROUP_new_curve_GF2m 000000018000b798     <common>
 0003:000007a0       OSSL_EC_GROUP_new_curve_GFp 000000018000b7a0     <common>
 0003:000007a8       OSSL_BN_CTX_new            000000018000b7a8     <common>
 0003:000007b0       OSSL_EC_KEY_set_private_key 000000018000b7b0     <common>
 0003:000007b8       OSSL_EC_KEY_set_public_key_affine_coordinates 000000018000b7b8     <common>
 0003:000007c0       OSSL_EC_KEY_new            000000018000b7c0     <common>
 0003:000007c8       OSSL_EC_KEY_get0_public_key 000000018000b7c8     <common>
 0003:000007d0       OSSL_ECDH_compute_key      000000018000b7d0     <common>
 0003:000007d8       OSSL_EC_KEY_free           000000018000b7d8     <common>
 0003:000007e0       OSSL_EC_KEY_generate_key   000000018000b7e0     <common>
 0003:000007e8       OSSL_chacha20_poly1305     000000018000b7e8     <common>
 0003:000007f0       OSSL_chacha20              000000018000b7f0     <common>
 0003:000007f8       OSSL_BN_num_bits           000000018000b7f8     <common>
 0003:00000800       OSSL_BN_bn2bin             000000018000b800     <common>
 0003:00000808       OSSL_BN_free               000000018000b808     <common>
 0003:00000810       OSSL_BN_set_negative       000000018000b810     <common>
 0003:00000818       OSSL_BN_bin2bn             000000018000b818     <common>
 0003:00000820       OSSL_BN_new                000000018000b820     <common>
 0003:00000828       OSSL_RSA_private_encrypt   000000018000b828     <common>
 0003:00000830       OSSL_RSA_public_decrypt    000000018000b830     <common>
 0003:00000838       OSSL_RSA_free              000000018000b838     <common>
 0003:00000840       OSSL_RSA_set0_crt_params   000000018000b840     <common>
 0003:00000848       OSSL_RSA_set0_factors      000000018000b848     <common>
 0003:00000850       OSSL_RSA_set0_key          000000018000b850     <common>
 0003:00000858       OSSL_RSA_new               000000018000b858     <common>
 0003:00000860       OSSL_DecryptFinal          000000018000b860     <common>
 0003:00000868       OSSL_DecryptUpdate         000000018000b868     <common>
 0003:00000870       OSSL_DecryptInit_ex        000000018000b870     <common>
 0003:00000878       OSSL_CIPHER_CTX_ctrl       000000018000b878     <common>
 0003:00000880       OSSL_aes_256_gcm           000000018000b880     <common>
 0003:00000888       OSSL_aes_192_gcm           000000018000b888     <common>
 0003:00000890       OSSL_aes_128_gcm           000000018000b890     <common>
 0003:00000898       OSSL_CipherFinal_ex        000000018000b898     <common>
 0003:000008a0       OSSL_CipherUpdate          000000018000b8a0     <common>
 0003:000008a8       OSSL_CIPHER_CTX_set_padding 000000018000b8a8     <common>
 0003:000008b0       OSSL_CipherInit_ex         000000018000b8b0     <common>
 0003:000008b8       OSSL_aes_256_cbc           000000018000b8b8     <common>
 0003:000008c0       OSSL_aes_192_cbc           000000018000b8c0     <common>
 0003:000008c8       OSSL_aes_128_cbc           000000018000b8c8     <common>
 0003:000008d0       OSSL_CIPHER_CTX_free       000000018000b8d0     <common>
 0003:000008d8       OSSL_CIPHER_CTX_new        000000018000b8d8     <common>
 0003:000008e0       OSSL_MD_CTX_free           000000018000b8e0     <common>
 0003:000008e8       OSSL_MD_CTX_reset          000000018000b8e8     <common>
 0003:000008f0       OSSL_DigestFinal_ex        000000018000b8f0     <common>
 0003:000008f8       OSSL_DigestUpdate          000000018000b8f8     <common>
 0003:00000900       OSSL_MD_CTX_copy_ex        000000018000b900     <common>
 0003:00000908       OSSL_DigestInit_ex         000000018000b908     <common>
 0003:00000910       OSSL_MD_CTX_new            000000018000b910     <common>
 0003:00000918       OSSL_sha512_256            000000018000b918     <common>
 0003:00000920       OSSL_sha512_224            000000018000b920     <common>
 0003:00000928       OSSL_sha512                000000018000b928     <common>
 0003:00000930       OSSL_sha384                000000018000b930     <common>
 0003:00000938       OSSL_sha224                000000018000b938     <common>
 0003:00000940       OSSL_sha256                000000018000b940     <common>
 0003:00000948       OSSL_sha1                  000000018000b948     <common>
 0003:00000950       OSSL_md5                   000000018000b950     <common>
 0003:00000958       OSSL_get_error             000000018000b958     <common>
 0003:00000960       OSSL_error_string          000000018000b960     <common>
 0003:00000968       OSSL_error_string_n        000000018000b968     <common>
 0003:00000970       OSSL_ECGF2M                000000018000b970     <common>
 0003:00000978       __dyn_tls_init_callback    000000018000b978     <common>

 entry point at        0001:00005970

 Static symbols

 0000:ffff1000       .debug$S                   0000000180000000     jncrypto.exp
 0000:ffff1000       .debug$S                   0000000180000000     vcruntime:VCRUNTIME140.dll
 0000:ffff1000       .debug$S                   0000000180000000     vcruntime:VCRUNTIME140.dll
 0000:ffff1000       .debug$S                   0000000180000000     vcruntime:VCRUNTIME140.dll
 0000:ffff1000       .debug$S                   0000000180000000     vcruntime:VCRUNTIME140.dll
 0000:ffff1000       .debug$S                   0000000180000000     vcruntime:VCRUNTIME140.dll
 0000:ffff1000       .debug$S                   0000000180000000     vcruntime:VCRUNTIME140.dll
 0000:ffff1000       .debug$S                   0000000180000000     ucrt:api-ms-win-crt-heap-l1-1-0.dll
 0000:ffff1000       .debug$S                   0000000180000000     ucrt:api-ms-win-crt-heap-l1-1-0.dll
 0000:ffff1000       .debug$S                   0000000180000000     ucrt:api-ms-win-crt-runtime-l1-1-0.dll
 0000:ffff1000       .debug$S                   0000000180000000     ucrt:api-ms-win-crt-runtime-l1-1-0.dll
 0000:ffff1000       .debug$S                   0000000180000000     ucrt:api-ms-win-crt-runtime-l1-1-0.dll
 0000:ffff1000       .debug$S                   0000000180000000     ucrt:api-ms-win-crt-runtime-l1-1-0.dll
 0000:ffff1000       .debug$S                   0000000180000000     ucrt:api-ms-win-crt-runtime-l1-1-0.dll
 0000:ffff1000       .debug$S                   0000000180000000     ucrt:api-ms-win-crt-runtime-l1-1-0.dll
 0000:ffff1000       .debug$S                   0000000180000000     ucrt:api-ms-win-crt-runtime-l1-1-0.dll
 0000:ffff1000       .debug$S                   0000000180000000     ucrt:api-ms-win-crt-runtime-l1-1-0.dll
 0000:ffff1000       .debug$S                   0000000180000000     ucrt:api-ms-win-crt-runtime-l1-1-0.dll
 0000:ffff1000       .debug$S                   0000000180000000     ucrt:api-ms-win-crt-runtime-l1-1-0.dll
 0000:ffff1000       .debug$S                   0000000180000000     ucrt:api-ms-win-crt-runtime-l1-1-0.dll
 0000:ffff1000       .debug$S                   0000000180000000     ucrt:api-ms-win-crt-runtime-l1-1-0.dll
 0000:ffff1000       .debug$S                   0000000180000000     ucrt:api-ms-win-crt-stdio-l1-1-0.dll
 0000:ffff1000       .debug$S                   0000000180000000     ucrt:api-ms-win-crt-stdio-l1-1-0.dll
 0000:ffff1000       .debug$S                   0000000180000000     ucrt:api-ms-win-crt-stdio-l1-1-0.dll
 0000:ffff1000       .debug$S                   0000000180000000     ucrt:api-ms-win-crt-stdio-l1-1-0.dll
 0000:ffff1000       .debug$S                   0000000180000000     ucrt:api-ms-win-crt-string-l1-1-0.dll
 0000:ffff1000       .debug$S                   0000000180000000     ucrt:api-ms-win-crt-string-l1-1-0.dll
 0000:ffff1000       .debug$S                   0000000180000000     ucrt:api-ms-win-crt-string-l1-1-0.dll
 0000:ffff1000       .debug$S                   0000000180000000     ucrt:api-ms-win-crt-string-l1-1-0.dll
 0000:ffff1000       .debug$S                   0000000180000000     ucrt:api-ms-win-crt-string-l1-1-0.dll
 0000:ffff1000       .debug$S                   0000000180000000     kernel32:KERNEL32.dll
 0000:ffff1000       .debug$S                   0000000180000000     kernel32:KERNEL32.dll
 0000:ffff1000       .debug$S                   0000000180000000     kernel32:KERNEL32.dll
 0000:ffff1000       .debug$S                   0000000180000000     kernel32:KERNEL32.dll
 0000:ffff1000       .debug$S                   0000000180000000     kernel32:KERNEL32.dll
 0000:ffff1000       .debug$S                   0000000180000000     kernel32:KERNEL32.dll
 0000:ffff1000       .debug$S                   0000000180000000     kernel32:KERNEL32.dll
 0000:ffff1000       .debug$S                   0000000180000000     kernel32:KERNEL32.dll
 0000:ffff1000       .debug$S                   0000000180000000     kernel32:KERNEL32.dll
 0000:ffff1000       .debug$S                   0000000180000000     kernel32:KERNEL32.dll
 0000:ffff1000       .debug$S                   0000000180000000     kernel32:KERNEL32.dll
 0000:ffff1000       .debug$S                   0000000180000000     kernel32:KERNEL32.dll
 0000:ffff1000       .debug$S                   0000000180000000     kernel32:KERNEL32.dll
 0000:ffff1000       .debug$S                   0000000180000000     kernel32:KERNEL32.dll
 0000:ffff1000       .debug$S                   0000000180000000     kernel32:KERNEL32.dll
 0000:ffff1000       .debug$S                   0000000180000000     kernel32:KERNEL32.dll
 0000:ffff1000       .debug$S                   0000000180000000     kernel32:KERNEL32.dll
 0000:ffff1000       .debug$S                   0000000180000000     kernel32:KERNEL32.dll
 0000:ffff1000       .debug$S                   0000000180000000     kernel32:KERNEL32.dll
 0000:ffff1000       .debug$S                   0000000180000000     kernel32:KERNEL32.dll
 0000:ffff1000       .debug$S                   0000000180000000     kernel32:KERNEL32.dll
 0000:ffff1000       .debug$S                   0000000180000000     kernel32:KERNEL32.dll
 0000:ffff1000       .debug$S                   0000000180000000     kernel32:KERNEL32.dll
 0000:ffff1000       .debug$S                   0000000180000000     kernel32:KERNEL32.dll
 0000:ffff1000       .debug$S                   0000000180000000     kernel32:KERNEL32.dll
 0000:ffff1000       .debug$S                   0000000180000000     kernel32:KERNEL32.dll
 0000:ffff1000       .debug$S                   0000000180000000     kernel32:KERNEL32.dll
 0000:ffff1000       .debug$S                   0000000180000000     kernel32:KERNEL32.dll
 0001:00000000       ECEncodeGF2m               0000000180001000 f   NativeCrypto.obj
 0001:00000110       ECEncodeGFp                0000000180001110 f   NativeCrypto.obj
 0001:00004c6c       extractVersionToJlong      0000000180005c6c f   NativeCrypto.obj
 0001:00004d00       find_crypto_library        0000000180005d00 f   NativeCrypto.obj
 0001:00004ef4       getArrayFromBN             0000000180005ef4 f   NativeCrypto.obj
 0001:00004f78       get_crypto_library_version 0000000180005f78 f   NativeCrypto.obj
 0001:00005120       load_crypto_library        0000000180006120 f   NativeCrypto.obj
 0001:000051e4       printErrors                00000001800061e4 f   NativeCrypto.obj
 0001:0000541c       thread_setup               000000018000641c f   NativeCrypto.obj
 0001:00005528       win32_locking_callback     0000000180006528 f   NativeCrypto.obj
 0001:00005620       $$000000                   0000000180006620     MSVCRT:amdsecgs.obj
 0001:00005650       ?dllmain_crt_dispatch@@YAHQEAUHINSTANCE__@@KQEAX@Z 0000000180006650 f   MSVCRT:dll_dllmain.obj
 0001:000056a0       ?dllmain_crt_process_attach@@YAHQEAUHINSTANCE__@@QEAX@Z 00000001800066a0 f   MSVCRT:dll_dllmain.obj
 0001:000057b8       ?dllmain_crt_process_detach@@YAH_N@Z 00000001800067b8 f   MSVCRT:dll_dllmain.obj
 0001:0000583c       ?dllmain_dispatch@@YAHQEAUHINSTANCE__@@KQEAX@Z 000000018000683c f   MSVCRT:dll_dllmain.obj
 0001:00005ab8       capture_previous_context   0000000180006ab8 f   MSVCRT:gs_report.obj
 0001:00006370       $$000000                   0000000180007370     MSVCRT:guard_dispatch.obj
 0001:00006390       $$000000                   0000000180007390     MSVCRT:guard_xfg_dispatch.obj
 0001:000063a6       ?fin$0@?0??dllmain_crt_process_attach@@YAHQEAUHINSTANCE__@@QEAX@Z@4HA 00000001800073a6 f   MSVCRT:dll_dllmain.obj
 0001:000063bd       ?fin$0@?0??dllmain_crt_process_detach@@YAH_N@Z@4HA 00000001800073bd f   MSVCRT:dll_dllmain.obj
 0001:000063d6       ?fin$1@?0??dllmain_crt_process_detach@@YAH_N@Z@4HA 00000001800073d6 f   MSVCRT:dll_dllmain.obj
 0001:000063ea       ?filt$0@?0??dllmain_dispatch@@YAHQEAUHINSTANCE__@@KQEAX@Z@4HA 00000001800073ea f   MSVCRT:dll_dllmain.obj
 0001:00006420       __scrt_is_nonwritable_in_current_image$filt$0 0000000180007420 f   MSVCRT:utility.obj
 0002:00000230       ?bundledLibName@?1??find_crypto_library@@9@9 0000000180008230     NativeCrypto.obj
 0002:00000244       ?pathSuffix@?5??find_crypto_library@@9@9 0000000180008244     NativeCrypto.obj
 0002:00000250       ?libNames@?1??find_crypto_library@@9@9 0000000180008250     NativeCrypto.obj
 0002:00001100       GS_ExceptionPointers       0000000180009100     MSVCRT:gs_report.obj
 0002:00001640       $unwind$fprintf            0000000180009640     NativeCrypto.obj
 0002:00001640       $unwind$sscanf             0000000180009640     NativeCrypto.obj
 0002:0000164c       $unwind$printf             000000018000964c     NativeCrypto.obj
 0002:00001658       $unwind$JNI_OnUnload       0000000180009658     NativeCrypto.obj
 0002:00001658       $unwind$OSSL102_RSA_set0_factors 0000000180009658     NativeCrypto.obj
 0002:00001658       $unwind$find_crypto_library 0000000180009658     NativeCrypto.obj
 0002:00001658       $unwind$thread_setup       0000000180009658     NativeCrypto.obj
 0002:00001658       $unwind$_DllMainCRTStartup 0000000180009658     MSVCRT:dll_dllmain.obj
 0002:00001668       $unwind$Java_jdk_crypto_jniprovider_NativeCrypto_loadCrypto 0000000180009668     NativeCrypto.obj
 0002:0000168c       $unwind$Java_jdk_crypto_jniprovider_NativeCrypto_DigestCreateContext 000000018000968c     NativeCrypto.obj
 0002:0000168c       $unwind$Java_jdk_crypto_jniprovider_NativeCrypto_ECCreatePrivateKey 000000018000968c     NativeCrypto.obj
 0002:000016a4       $unwind$Java_jdk_crypto_jniprovider_NativeCrypto_DigestDestroyContext 00000001800096a4     NativeCrypto.obj
 0002:000016a4       $unwind$Java_jdk_crypto_jniprovider_NativeCrypto_DigestReset 00000001800096a4     NativeCrypto.obj
 0002:000016a4       $unwind$win32_locking_callback 00000001800096a4     NativeCrypto.obj
 0002:000016a4       $unwind$__raise_securityfailure 00000001800096a4     MSVCRT:gs_report.obj
 0002:000016a4       $unwind$__scrt_initialize_crt 00000001800096a4     MSVCRT:utility.obj
 0002:000016a4       $unwind$__scrt_initialize_onexit_tables 00000001800096a4     MSVCRT:utility.obj
 0002:000016a4       $unwind$__scrt_release_startup_lock 00000001800096a4     MSVCRT:utility.obj
 0002:000016a4       $unwind$__scrt_uninitialize_crt 00000001800096a4     MSVCRT:utility.obj
 0002:000016ac       $unwind$Java_jdk_crypto_jniprovider_NativeCrypto_DigestUpdate 00000001800096ac     NativeCrypto.obj
 0002:000016ac       $unwind$getArrayFromBN     00000001800096ac     NativeCrypto.obj
 0002:000016ac       $unwind$get_crypto_library_version 00000001800096ac     NativeCrypto.obj
 0002:000016c4       $unwind$Java_jdk_crypto_jniprovider_NativeCrypto_DigestComputeAndReset 00000001800096c4     NativeCrypto.obj
 0002:000016d8       $unwind$Java_jdk_crypto_jniprovider_NativeCrypto_CreateContext 00000001800096d8     NativeCrypto.obj
 0002:000016d8       $unwind$Java_jdk_crypto_jniprovider_NativeCrypto_DestroyContext 00000001800096d8     NativeCrypto.obj
 0002:000016d8       $unwind$Java_jdk_crypto_jniprovider_NativeCrypto_ECDestroyKey 00000001800096d8     NativeCrypto.obj
 0002:000016d8       $unwind$Java_jdk_crypto_jniprovider_NativeCrypto_destroyRSAKey 00000001800096d8     NativeCrypto.obj
 0002:000016d8       $unwind$__scrt_initialize_default_local_stdio_options 00000001800096d8     MSVCRT:default_local_stdio_options.obj
 0002:000016d8       $unwind$?dllmain_crt_dispatch@@YAHQEAUHINSTANCE__@@KQEAX@Z 00000001800096d8     MSVCRT:dll_dllmain.obj
 0002:000016d8       $unwind$DllMain            00000001800096d8     MSVCRT:dll_dllmain_stub.obj
 0002:000016d8       $unwind$__GSHandlerCheck   00000001800096d8     MSVCRT:gshandler.obj
 0002:000016d8       $unwind$__scrt_acquire_startup_lock 00000001800096d8     MSVCRT:utility.obj
 0002:000016d8       $unwind$__scrt_dllmain_after_initialize_c 00000001800096d8     MSVCRT:utility.obj
 0002:000016d8       $unwind$__scrt_dllmain_before_initialize_c 00000001800096d8     MSVCRT:utility.obj
 0002:000016d8       $unwind$__scrt_dllmain_crt_thread_attach 00000001800096d8     MSVCRT:utility.obj
 0002:000016d8       $unwind$__scrt_dllmain_crt_thread_detach 00000001800096d8     MSVCRT:utility.obj
 0002:000016d8       $unwind$__scrt_dllmain_uninitialize_c 00000001800096d8     MSVCRT:utility.obj
 0002:000016d8       $unwind$__scrt_dllmain_uninitialize_critical 00000001800096d8     MSVCRT:utility.obj
 0002:000016e0       $unwind$Java_jdk_crypto_jniprovider_NativeCrypto_CBCInit 00000001800096e0     NativeCrypto.obj
 0002:000016fc       $unwind$Java_jdk_crypto_jniprovider_NativeCrypto_CBCUpdate 00000001800096fc     NativeCrypto.obj
 0002:00001710       $unwind$Java_jdk_crypto_jniprovider_NativeCrypto_CBCFinalEncrypt 0000000180009710     NativeCrypto.obj
 0002:00001730       $unwind$Java_jdk_crypto_jniprovider_NativeCrypto_GCMDecrypt 0000000180009730     NativeCrypto.obj
 0002:00001730       $unwind$Java_jdk_crypto_jniprovider_NativeCrypto_GCMEncrypt 0000000180009730     NativeCrypto.obj
 0002:00001748       $unwind$Java_jdk_crypto_jniprovider_NativeCrypto_createRSAPublicKey 0000000180009748     NativeCrypto.obj
 0002:00001760       $unwind$Java_jdk_crypto_jniprovider_NativeCrypto_createRSAPrivateCrtKey 0000000180009760     NativeCrypto.obj
 0002:00001778       $unwind$Java_jdk_crypto_jniprovider_NativeCrypto_RSADP 0000000180009778     NativeCrypto.obj
 0002:00001790       $unwind$Java_jdk_crypto_jniprovider_NativeCrypto_ECDeriveKey 0000000180009790     NativeCrypto.obj
 0002:00001790       $unwind$Java_jdk_crypto_jniprovider_NativeCrypto_RSAEP 0000000180009790     NativeCrypto.obj
 0002:000017a8       $unwind$Java_jdk_crypto_jniprovider_NativeCrypto_ChaCha20Init 00000001800097a8     NativeCrypto.obj
 0002:000017c0       $unwind$Java_jdk_crypto_jniprovider_NativeCrypto_ChaCha20Update 00000001800097c0     NativeCrypto.obj
 0002:000017d8       $unwind$Java_jdk_crypto_jniprovider_NativeCrypto_ChaCha20FinalEncrypt 00000001800097d8     NativeCrypto.obj
 0002:000017ec       $unwind$Java_jdk_crypto_jniprovider_NativeCrypto_ChaCha20FinalDecrypt 00000001800097ec     NativeCrypto.obj
 0002:00001804       $unwind$Java_jdk_crypto_jniprovider_NativeCrypto_ECGenerateKeyPair 0000000180009804     NativeCrypto.obj
 0002:0000181c       $unwind$Java_jdk_crypto_jniprovider_NativeCrypto_ECCreatePublicKey 000000018000981c     NativeCrypto.obj
 0002:00001838       $unwind$Java_jdk_crypto_jniprovider_NativeCrypto_ECEncodeGF 0000000180009838     NativeCrypto.obj
 0002:00001850       $unwind$Java_jdk_crypto_jniprovider_NativeCrypto_PBEDerive 0000000180009850     NativeCrypto.obj
 0002:00001850       $unwind$Java_jdk_crypto_jniprovider_NativeCrypto_PBKDF2Derive 0000000180009850     NativeCrypto.obj
 0002:0000186c       $unwind$Java_jdk_crypto_jniprovider_NativeCrypto_ECDSASign 000000018000986c     NativeCrypto.obj
 0002:00001888       $unwind$Java_jdk_crypto_jniprovider_NativeCrypto_ECDSAVerify 0000000180009888     NativeCrypto.obj
 0002:000018a4       $unwind$Java_jdk_crypto_jniprovider_NativeCrypto_XDHCreateKeys 00000001800098a4     NativeCrypto.obj
 0002:000018c0       $unwind$Java_jdk_crypto_jniprovider_NativeCrypto_XDHGenerateSecret 00000001800098c0     NativeCrypto.obj
 0002:000018d8       $unwind$OSSL102_RSA_set0_crt_params 00000001800098d8     NativeCrypto.obj
 0002:000018d8       $unwind$OSSL102_RSA_set0_key 00000001800098d8     NativeCrypto.obj
 0002:000018d8       $unwind$__scrt_dllmain_exception_filter 00000001800098d8     MSVCRT:utility.obj
 0002:000018ec       $unwind$setECPublicKey     00000001800098ec     NativeCrypto.obj
 0002:00001908       $unwind$printErrors        0000000180009908     NativeCrypto.obj
 0002:00001918       $unwind$extractVersionToJlong 0000000180009918     NativeCrypto.obj
 0002:00001924       $unwind$load_crypto_library 0000000180009924     NativeCrypto.obj
 0002:00001934       $unwind$convertJavaBItoBN  0000000180009934     NativeCrypto.obj
 0002:00001934       $unwind$_RTC_Initialize    0000000180009934     MSVCRT:initsect.obj
 0002:00001934       $unwind$_RTC_Terminate     0000000180009934     MSVCRT:initsect.obj
 0002:00001940       $unwind$ECEncodeGF2m       0000000180009940     NativeCrypto.obj
 0002:00001940       $unwind$ECEncodeGFp        0000000180009940     NativeCrypto.obj
 0002:00001958       $unwind$__GSHandlerCheckCommon 0000000180009958     MSVCRT:gshandler.obj
 0002:00001960       $xdatasym                  0000000180009960     MSVCRT:amdsecgs.obj
 0002:00001964       $unwind$?dllmain_crt_process_attach@@YAHQEAUHINSTANCE__@@QEAX@Z 0000000180009964     MSVCRT:dll_dllmain.obj
 0002:000019a0       $unwind$?fin$0@?0??dllmain_crt_process_attach@@YAHQEAUHINSTANCE__@@QEAX@Z@4HA 00000001800099a0     MSVCRT:dll_dllmain.obj
 0002:000019a0       $unwind$?fin$0@?0??dllmain_crt_process_detach@@YAH_N@Z@4HA 00000001800099a0     MSVCRT:dll_dllmain.obj
 0002:000019a0       $unwind$?fin$1@?0??dllmain_crt_process_detach@@YAH_N@Z@4HA 00000001800099a0     MSVCRT:dll_dllmain.obj
 0002:000019a8       $unwind$?dllmain_crt_process_detach@@YAH_N@Z 00000001800099a8     MSVCRT:dll_dllmain.obj
 0002:000019fc       $unwind$?dllmain_dispatch@@YAHQEAUHINSTANCE__@@KQEAX@Z 00000001800099fc     MSVCRT:dll_dllmain.obj
 0002:00001a24       $unwind$?filt$0@?0??dllmain_dispatch@@YAHQEAUHINSTANCE__@@KQEAX@Z@4HA 0000000180009a24     MSVCRT:dll_dllmain.obj
 0002:00001a2c       $unwind$__report_gsfailure 0000000180009a2c     MSVCRT:gs_report.obj
 0002:00001a34       $unwind$capture_previous_context 0000000180009a34     MSVCRT:gs_report.obj
 0002:00001a40       $unwind$__security_init_cookie 0000000180009a40     MSVCRT:gs_support.obj
 0002:00001a4c       $unwind$__scrt_is_nonwritable_in_current_image 0000000180009a4c     MSVCRT:utility.obj
 0002:00001a6c       $unwind$__scrt_is_nonwritable_in_current_image$filt$0 0000000180009a6c     MSVCRT:utility.obj
 0002:00001a74       $unwind$__scrt_fastfail    0000000180009a74     MSVCRT:utility_desktop.obj
 0002:00001a84       $unwind$__isa_available_init 0000000180009a84     MSVCRT:cpu_disp.obj
 0002:00001a98       $xdatasym                  0000000180009a98     MSVCRT:guard_dispatch.obj
 0002:00001aa0       $xdatasym                  0000000180009aa0     MSVCRT:guard_xfg_dispatch.obj
 0002:00001ab0       .edata                     0000000180009ab0     jncrypto.exp
 0002:00001ad8       rgpv                       0000000180009ad8     jncrypto.exp
 0002:00001b70       rgszName                   0000000180009b70     jncrypto.exp
 0002:00001c08       rgwOrd                     0000000180009c08     jncrypto.exp
 0002:00001c54       szName                     0000000180009c54     jncrypto.exp
 0002:00001c61       $N00001                    0000000180009c61     jncrypto.exp
 0002:00001c6e       $N00002                    0000000180009c6e     jncrypto.exp
 0002:00001ca7       $N00003                    0000000180009ca7     jncrypto.exp
 0002:00001cd8       $N00004                    0000000180009cd8     jncrypto.exp
 0002:00001d0b       $N00005                    0000000180009d0b     jncrypto.exp
 0002:00001d49       $N00006                    0000000180009d49     jncrypto.exp
 0002:00001d87       $N00007                    0000000180009d87     jncrypto.exp
 0002:00001dbd       $N00008                    0000000180009dbd     jncrypto.exp
 0002:00001df5       $N00009                    0000000180009df5     jncrypto.exp
 0002:00001e2c       $N00010                    0000000180009e2c     jncrypto.exp
 0002:00001e64       $N00011                    0000000180009e64     jncrypto.exp
 0002:00001ea3       $N00012                    0000000180009ea3     jncrypto.exp
 0002:00001ee0       $N00013                    0000000180009ee0     jncrypto.exp
 0002:00001f1e       $N00014                    0000000180009f1e     jncrypto.exp
 0002:00001f53       $N00015                    0000000180009f53     jncrypto.exp
 0002:00001f89       $N00016                    0000000180009f89     jncrypto.exp
 0002:00001fc5       $N00017                    0000000180009fc5     jncrypto.exp
 0002:00002000       $N00018                    000000018000a000     jncrypto.exp
 0002:00002033       $N00019                    000000018000a033     jncrypto.exp
 0002:00002068       $N00020                    000000018000a068     jncrypto.exp
 0002:0000209d       $N00021                    000000018000a09d     jncrypto.exp
 0002:000020d3       $N00022                    000000018000a0d3     jncrypto.exp
 0002:00002107       $N00023                    000000018000a107     jncrypto.exp
 0002:00002142       $N00024                    000000018000a142     jncrypto.exp
 0002:00002178       $N00025                    000000018000a178     jncrypto.exp
 0002:000021ac       $N00026                    000000018000a1ac     jncrypto.exp
 0002:000021e0       $N00027                    000000018000a1e0     jncrypto.exp
 0002:00002213       $N00028                    000000018000a213     jncrypto.exp
 0002:00002249       $N00029                    000000018000a249     jncrypto.exp
 0002:00002278       $N00030                    000000018000a278     jncrypto.exp
 0002:000022a7       $N00031                    000000018000a2a7     jncrypto.exp
 0002:000022de       $N00032                    000000018000a2de     jncrypto.exp
 0002:00002319       $N00033                    000000018000a319     jncrypto.exp
 0002:00002359       $N00034                    000000018000a359     jncrypto.exp
 0002:00002395       $N00035                    000000018000a395     jncrypto.exp
 0002:000023cc       $N00036                    000000018000a3cc     jncrypto.exp
 0002:00002404       $N00037                    000000018000a404     jncrypto.exp
 0002:0000243b       $N00038                    000000018000a43b     jncrypto.exp
 0002:000028d6       .idata$6                   000000018000a8d6     kernel32:KERNEL32.dll
 0002:00002926       .idata$6                   000000018000a926     vcruntime:VCRUNTIME140.dll
 0002:00002a72       .idata$6                   000000018000aa72     ucrt:api-ms-win-crt-string-l1-1-0.dll
 0002:00002a94       .idata$6                   000000018000aa94     ucrt:api-ms-win-crt-stdio-l1-1-0.dll
 0002:00002ab4       .idata$6                   000000018000aab4     ucrt:api-ms-win-crt-heap-l1-1-0.dll
 0002:00002ad4       .idata$6                   000000018000aad4     ucrt:api-ms-win-crt-runtime-l1-1-0.dll
 0003:00000044       OSSL_IS_FIPS               000000018000b044     NativeCrypto.obj
 0003:00000048       OSSL_CRYPTO_num_locks      000000018000b048     NativeCrypto.obj
 0003:00000050       OSSL_CRYPTO_THREADID_set_numeric 000000018000b050     NativeCrypto.obj
 0003:00000058       OSSL_OPENSSL_malloc        000000018000b058     NativeCrypto.obj
 0003:00000060       OSSL_OPENSSL_free          000000018000b060     NativeCrypto.obj
 0003:00000068       OSSL_CRYPTO_THREADID_set_callback 000000018000b068     NativeCrypto.obj
 0003:00000070       OSSL_CRYPTO_set_locking_callback 000000018000b070     NativeCrypto.obj
 0003:00000078       crypto_library             000000018000b078     NativeCrypto.obj
 0003:00000080       lock_cs                    000000018000b080     NativeCrypto.obj
 0003:00000088       ?__proc_attached@@3HA      000000018000b088     MSVCRT:dll_dllmain.obj
 0003:00000090       GS_ExceptionRecord         000000018000b090     MSVCRT:gs_report.obj
 0003:00000130       GS_ContextRecord           000000018000b130     MSVCRT:gs_report.obj
 0003:00000620       ?is_initialized_as_dll@@3_NA 000000018000b620     MSVCRT:utility.obj
 0003:00000621       ?module_local_atexit_table_initialized@@3_NA 000000018000b621     MSVCRT:utility.obj
 0003:00000628       ?module_local_atexit_table@@3U_onexit_table_t@@A 000000018000b628     MSVCRT:utility.obj
 0003:00000640       ?module_local_at_quick_exit_table@@3U_onexit_table_t@@A 000000018000b640     MSVCRT:utility.obj
 0005:00000060       $R000000                   000000018000d060     jncrypto.dll.res
